:020000040000FA
:040000008A01032846
:0A00060083120313981383160313EB
:1000100007309C009D019B0185018601831203131B
:100020003820152020202C20142830308400103057
:10003000A300230861208000840AA30B192808006C
:10004000803041200830A2003F30840000084D205D
:100050008403A20B26280800C03041200830A200EB
:100060003730840000084D208403A20B322808009A
:100070003830412001304120033041200F304120F1
:100080000800860059200430850059200030850082
:100090005920043085005920080086005920063078
:1000A00085005920023085005920063085005920EE
:1000B00008006430A100A000A00B5C28A10B5B2805
:1000C000080082072034453456344F344C345534BC
:1000D00050344934433420342034313436344634B7
:0800E000383438342034203498
:00000001FF
